:020000040000FA
:04000000CD303A289D
:040004000034003490
:08000800A000030EA100831209
:100010008B1C32288B1032181428B21C3228643002
:10002000010203183128182800001628172818285C
:1000300019281A281B281C281D281E281F283210A2
:10004000B214A810031005190314AA0DA90DA80DC8
:10005000B10B322832152A08AF002908AE00280853
:10006000AD00B21081010B11210E8300A00E200EF5
:02007000090085
:0C007400203084008001840A80300402E7
:10008000031C3C281230B100FC2183160C3085057E
:1000900087018312850187010730990000309A009B
:1000A000103083168E008312603083168F00831207
:1000B0000030831691009F008312C83083168100A0
:1000C000831231309000003083168C008312103080
:1000D0008B00BD1B7128851971286400851D6D2852
:1000E0002B230E2381018E018F010B118B100B101E
:1000F0008C018B17892032199F20B40B872803109D
:1001000085190314BA0DF0303A02031957217123EF
:100110007A286400321808000B1D08000B11B21079
:1001200032141230B100051D9A28331483160113BE
:10013000831208003310831601178312080032114E
:100140000130B7008B132030370783169B001C1437
:100150001A088312A400A500C030A5061030370786
:1001600083169B001C141A088312A3000030370763
:1001700083169B001C141A088312A2008B17331CD1
:10018000C72822090339A200A309A409A509220846
:100190002D02031D512923082E02031D5129240875
:1001A0002F02031D512901303702031DDC283E18A0
:1001B000DC283E143F141E2202303702031DE528BE
:1001C000BE18E528BE143F142D2203303702031D4C
:1001D000EE283E19EE283E153F143922043037022E
:1001E000031DF728BE19F728BE153F144522053018
:1001F0003702031D00293E1A00293E163F145122E2
:1002000006303702031D0929BE1A0929BE163F14FC
:100210005D2207303702031D12293E1B12293E17AB
:100220003F146C2208303702031D1B29BE1B1B29FB
:10023000BE173F147B2209303702031D24295E18A4
:1002400024295E143F1486220A303702031D2D290B
:10025000DE182D29DE143F1491220B303702031DC6
:1002600036295E1936295E153F149C220C30370260
:10027000031D3F29DE193F29DE153F14A7220D304B
:100280003702031D48295E1A48295E163F14B22220
:100290000E303702031D5129DE1A5129DE163F1494
:1002A000BD22B70A0F30370203180800A228013018
:1002B000B600B400B500B70085018701B2138920EC
:1002C000B40B6F29031085190314BA0DF0303A02EC
:1002D00003199629B50B6F299630B500A021321D60
:1002E0005F293211331C79292D090339AD00AE097C
:1002F000AF092F1CB2132F1C5F29B21B5F292E18C8
:100300005F29B2178B1320303707BC002F08BB00C2
:10031000E72110303707BC002E08BB00E721003072
:100320003707BC002D08BB00E7218B17850187012B
:10033000B70AB6010F303702031C5F290E230800ED
:10034000013037020319C822023037020319CD22C7
:10035000033037020319D222043037020319D7229F
:10036000053037020319DC22063037020319E12277
:10037000073037020319E622083037020319EB224F
:10038000093037020319F0220A3037020319F52227
:100390000B3037020319FA220C3037020319FF22FF
:1003A0000D303702031904230E30370203190923D5
:1003B00008003F1C08003F101030BC003E08BB0086
:1003C000E7213030BC005E08BB00E72108008B133A
:1003D0003B0883161C159A0083123C0883169B0069
:1003E00055309D00AA309D009C1464009C18F5298E
:1003F0001C1183128B170800831600309B001C14FD
:100400001A088312BD00831610309B001C141A08B2
:100410008312BE00831630309B001C141A0883120E
:10042000DE00FF30C800CA15CB15CC15CD15CE1592
:10043000CF15D015D115D215D31508008130BE05C2
:10044000FF30DE054130C405C0000030C200C600E8
:10045000BD185F14BD18DF1408008230BE05FF30E0
:10046000DE058030C405C0000030C200C6005F1049
:1004700008008430BE05FF30DE054230C405C000F0
:100480004030C200C6005F1008008830BE05FF3053
:10049000DE054630C405C0004030C200C6005F1013
:1004A00008009030BE05FF30DE058A30C405C0006C
:1004B0008030C200C6005F100800A030BE05FF30CB
:1004C000DE055130C405C0001030C200C600BD18A2
:1004D0005F14BD18DF140800C030BE05FF30DE0514
:1004E0007130C405C0000030C200C600BD185F14E2
:1004F000BD18DF140800FF30BE05C030DE054030F7
:10050000C505C1000030C300C70008007F30BE052C
:10051000C130DE058030C505C1000030C300C70012
:1005200008007F30BE05C230DE054030C505C10081
:100530004030C300C70008007F30BE05C430DE0570
:100540004030C505C1004030C300C70008007F30FF
:10055000BE05C830DE058030C505C1008030C3004F
:10056000C70008007F30BE05D030DE054030C5052D
:10057000C1000030C300C70008007F30BE05E03076
:10058000DE054030C505C1000030C300C7000800CB
:10059000103085060130870608003330850620308C
:1005A00087060800203085060130870608002130C4
:1005B0008506013087060800223085062030870630
:1005C00008001030850603308706080010308506C5
:1005D00007308706080000308506103087060800BF
:1005E0000030850608308706080000308506103088
:1005F00087060800003085061030870608000030A6
:10060000850608308706080000308506103087060A
:100610000800003085061030870608003E181E22AC
:10062000BE182D223E193922BE1945223E1A5122EA
:10063000BE1A5D223E1B6C22BE1B7B225E188622E8
:10064000DE1891225E199C22DE19A7225E1AB222C0
:10065000DE1ABD220800B601B401B5013D1C332BE2
:10066000BD01BD14352BBD013D143D08B60064002D
:10067000392B3A2B3B2B3C2B3D2BFF30B51B8500F8
:10068000B51F8501B40B372BB50B372B0310B60CF8
:10069000B608031D372B0030BC003D08BB00E72126
:1006A000080005125C180516DC1C8512DC1885167E
:1006B0005C1D05105C190514DC1D8510DC19851402
:1006C0005C1E87105C1A8714DC1E0711DC1A0715E4
:1006D0005C1F07105C1B0714DC1F8712DC1B8716CE
:1006E00008008F08031908008F0178308E00C80FAA
:1006F0009F2DC80A441CA12B461C922BCA1C832B7D
:10070000CA014A15AF2B4A1D882BCA01CA15AF2B47
:10071000CA1D8D2BCA014A16AF2B4A1EAF2BCA0128
:10072000CA14AF2B4A1D972BCA014A16AF2BCA1DFC
:100730009C2BCA014A16AF2B4A1EAF2BCA01CA1402
:10074000AF2BCA1CA62BCA014A15AF2B4A1DAB2BD7
:10075000CA01CA15AF2B4A1EAF2BCA014A15C41CC9
:10076000D62BC61CC72BCB1CB82BCB014B15E42BAF
:100770004B1DBD2BCB01CB15E42BCB1DC22BCB01CD
:100780004B16E42B4B1EE42BCB01CB14E42B4B1D5F
:10079000CC2BCB014B16E42BCB1DD12BCB014B1615
:1007A000E42B4B1EE42BCB01CB14E42BCB1CDB2B1B
:1007B000CB014B15E42B4B1DE02BCB01CB15E42BD0
:1007C0004B1EE42BCB014B15441D0B2C461DFC2B63
:1007D000CC1CED2BCC014C15192C4C1DF22BCC0153
:1007E000CC15192CCC1DF72BCC014C16192C4C1EFA
:1007F000192CCC01CC14192C4C1D012CCC014C16FD
:10080000192CCC1D062CCC014C16192C4C1E192C65
:10081000CC01CC14192CCC1C102CCC014C15192C4F
:100820004C1D152CCC01CC15192C4C1E192CCC01AF
:100830004C15C41D412CC61D322CCD1C232CCD01C2
:100840004D155F134F2C4D1D282CCD01CD154F2C70
:10085000CD1D2D2CCD014D164F2C4D1E4F2CCD01F5
:10086000CD144F2C4D1D372CCD014D164F2CCD1DC9
:100870003C2CCD014D164F2C4D1E4F2CCD01CD14CF
:100880004F2CCD1C462CCD014D154F2C4D1D4B2C06
:10089000CD01CD154F2C4D1E4F2CCD014D155F1B9D
:1008A000782C441E782C461E692CCE1C5A2CCE0166
:1008B0004E15862C4E1D5F2CCE01CE15862CCE1DDE
:1008C000642CCE014E16862C4E1E862CCE01CE14E4
:1008D000862C4E1D6E2CCE014E16862CCE1D732CF2
:1008E000CE014E16862C4E1E862CCE01CE14862CA2
:1008F000CE1C7D2CCE014E15862C4E1D822CCE0199
:10090000CE15862C4E1E862CCE014E15C41EAD2C47
:10091000C61E9E2CCF1C8F2CCF014F15BB2C4F1DFC
:10092000942CCF01CF15BB2CCF1D992CCF014F1686
:10093000BB2C4F1EBB2CCF01CF14BB2C4F1DA32CA7
:10094000CF014F16BB2CCF1DA82CCF014F16BB2CAF
:100950004F1EBB2CCF01CF14BB2CCF1CB22CCF0110
:100960004F15BB2C4F1DB72CCF01CF15BB2C4F1EE5
:10097000BB2CCF014F15441FE22C461FD32CD01C9B
:10098000C42CD0015015F02C501DC92CD001D0150D
:10099000F02CD01DCE2CD0015016F02C501EF02C77
:1009A000D001D014F02C501DD82CD0015016F02CB2
:1009B000D01DDD2CD0015016F02C501EF02CD00193
:1009C000D014F02CD01CE72CD0015015F02C501D69
:1009D000EC2CD001D015F02C501EF02CD00150156D
:1009E000C41F172DC61F082DD11CF92CD10151157C
:1009F000252D511DFE2CD101D115252DD11D032DE5
:100A0000D1015116252D511E252DD101D114252D91
:100A1000511D0D2DD1015116252DD11D122DD101A4
:100A20005116252D511E252DD101D114252DD11C56
:100A30001C2DD1015115252D511D212DD101D1156F
:100A4000252D511E252DD1015115DF184F2D451F84
:100A50004F2D471F402DD21C312DD2015215DF13CF
:100A60005D2D521D362DD201D2155D2DD21D3B2D8F
:100A7000D20152165D2D521E5D2DD201D2145D2D74
:100A8000521D452DD20152165D2DD21D4A2DD20187
:100A900052165D2D521E5D2DD201D2145D2DD21C39
:100AA000542DD20152155D2D521D592DD201D21552
:100AB0005D2D521E5D2DD2015215DF18882DDF1BD2
:100AC000882DC51F882DC71F792DD31C6A2DD301F2
:100AD0005315962D531D6F2DD301D315962DD31D70
:100AE000742DD3015316962D531E962DD301D31476
:100AF000962D531D7E2DD3015316962DD31D832D78
:100B0000D3015316962D531E962DD301D314962D33
:100B1000D31C8D2DD3015315962D531D922DD3012A
:100B2000D315962D531E962DD3015315D921400868
:100B3000C4004108C5005F18DF145F1CDF104808BF
:100B4000C9000C304A05031D05120C304B05031D6E
:100B500085120C304C05031D05100C304D05031D8E
:100B600085100C304E05031D87100C304F05031DFA
:100B700007110C305005031D07100C305105031DE3
:100B800087120C305205031D07120C305305031D4C
:100B9000871149080E020318F92D12304A05031D6A
:100BA000051612304B05031D851612304C05031D2A
:100BB000051412304D05031D851412304E05031D1A
:100BC000871412304F05031D071512305005031D01
:100BD000071412305105031D871612305205031DEC
:100BE000071612305305031D8715FF3048020319FD
:100BF00008008F08031D0800892049080E02031C05
:100C0000F92D18304A05031D051206304A05031D4B
:100C1000051618304B05031D851206304B05031DC4
:100C2000851618304C05031D051006304C05031DB4
:100C3000051418304D05031D851006304D05031DA4
:100C4000851418304E05031D871006304E05031D10
:100C5000871418304F05031D071106304F05031D7B
:100C6000071518305005031D071006305005031DE9
:100C7000071418305105031D871206305105031D56
:100C8000871618305205031D071206305205031D42
:100C9000071618305305031D871106305305031D31
:040CA00087150800AC
:084000000500030006000900A1
:02400E00CC33B1
:10420000010003000300030003000200020002009B
:104210000200000000000000000003000300FF0097
:10422000810000000000000000000000000000000D
:104230000000C000C000C000C000C000C000FF00FF
:10424000FF00C300F300CF00FF00C300F300CF0066
:10425000FF00C300F300CF00FF00C300F300FF0026
:104260000000FF00FF00FF00FF00FF00FF00FF0055
:10427000FF00FF00FF00FF00FF00FF00FF00FF0046
:10428000FF00FF00FF00FF00FF00FF00FF00FF0036
:10429000FF00FF00FF00FF00FF00FF00FF00FF0026
:1042A000FF00FF00FF00FF00FF00FF00FF00FF0016
:1042B000FF00FF00FF00FF00FF00FF00FF00FF0006
:1042C000FF00FF00FF00FF00FF00FF00FF00FF00F6
:1042D000FF00FF00FF00FF00FF00FF00FF00FF00E6
:1042E000FF00FF00FF00FF00FF00FF00FF00FF00D6
:1042F000FF00FF00FF00FF00FF00FF00FF00AA001B
:00000001FF
